


ARM Macro Assembler    Page 1 


    1 00000000         ;******************** (C) COPYRIGHT 2011 STMicroelectron
                       ics ********************
    2 00000000         ;* File Name          : startup_stm32f10x_hd.s
    3 00000000         ;* Author             : MCD Application Team
    4 00000000         ;* Version            : V3.5.0
    5 00000000         ;* Date               : 11-March-2011
    6 00000000         ;* Description        : STM32F10x High Density Devices v
                       ector table for MDK-ARM 
    7 00000000         ;*                      toolchain. 
    8 00000000         ;*                      This module performs:
    9 00000000         ;*                      - Set the initial SP
   10 00000000         ;*                      - Set the initial PC == Reset_Ha
                       ndler
   11 00000000         ;*                      - Set the vector table entries w
                       ith the exceptions ISR address
   12 00000000         ;*                      - Configure the clock system and
                        also configure the external 
   13 00000000         ;*                        SRAM mounted on STM3210E-EVAL 
                       board to be used as data 
   14 00000000         ;*                        memory (optional, to be enable
                       d by user)
   15 00000000         ;*                      - Branches to __main in the C li
                       brary (which eventually
   16 00000000         ;*                        calls main()).
   17 00000000         ;*                      After Reset the CortexM3 process
                       or is in Thread mode,
   18 00000000         ;*                      priority is Privileged, and the 
                       Stack is set to Main.
   19 00000000         ;* <<< Use Configuration Wizard in Context Menu >>>   
   20 00000000         ;*******************************************************
                       ************************
   21 00000000         ; THE PRESENT FIRMWARE WHICH IS FOR GUIDANCE ONLY AIMS A
                       T PROVIDING CUSTOMERS
   22 00000000         ; WITH CODING INFORMATION REGARDING THEIR PRODUCTS IN OR
                       DER FOR THEM TO SAVE TIME.
   23 00000000         ; AS A RESULT, STMICROELECTRONICS SHALL NOT BE HELD LIAB
                       LE FOR ANY DIRECT,
   24 00000000         ; INDIRECT OR CONSEQUENTIAL DAMAGES WITH RESPECT TO ANY 
                       CLAIMS ARISING FROM THE
   25 00000000         ; CONTENT OF SUCH FIRMWARE AND/OR THE USE MADE BY CUSTOM
                       ERS OF THE CODING
   26 00000000         ; INFORMATION CONTAINED HEREIN IN CONNECTION WITH THEIR 
                       PRODUCTS.
   27 00000000         ;*******************************************************
                       ************************
   28 00000000         
   29 00000000         ; Amount of memory (in bytes) allocated for Stack
   30 00000000         ; Tailor this value to your application needs
   31 00000000         ; <h> Stack Configuration
   32 00000000         ;   <o> Stack Size (in Bytes) <0x0-0xFFFFFFFF:8>
   33 00000000         ; </h>
   34 00000000         
   35 00000000                 IMPORT           WWDG_IRQHandler
   36 00000000                 IMPORT           PVD_IRQHandler
   37 00000000                 IMPORT           TAMPER_IRQHandler
   38 00000000                 IMPORT           RTC_IRQHandler
   39 00000000                 IMPORT           FLASH_IRQHandler
   40 00000000                 IMPORT           RCC_IRQHandler
   41 00000000                 IMPORT           EXTI0_IRQHandler



ARM Macro Assembler    Page 2 


   42 00000000                 IMPORT           EXTI1_IRQHandler
   43 00000000                 IMPORT           EXTI2_IRQHandler
   44 00000000                 IMPORT           EXTI3_IRQHandler
   45 00000000                 IMPORT           EXTI4_IRQHandler
   46 00000000                 IMPORT           DMA1_Channel1_IRQHandler
   47 00000000                 IMPORT           DMA1_Channel2_IRQHandler
   48 00000000                 IMPORT           DMA1_Channel3_IRQHandler
   49 00000000                 IMPORT           DMA1_Channel4_IRQHandler
   50 00000000                 IMPORT           DMA1_Channel5_IRQHandler
   51 00000000                 IMPORT           DMA1_Channel6_IRQHandler
   52 00000000                 IMPORT           DMA1_Channel7_IRQHandler
   53 00000000                 IMPORT           ADC1_2_IRQHandler
   54 00000000                 IMPORT           USB_HP_CAN1_TX_IRQHandler
   55 00000000                 IMPORT           USB_LP_CAN1_RX0_IRQHandler
   56 00000000                 IMPORT           CAN1_RX1_IRQHandler
   57 00000000                 IMPORT           CAN1_SCE_IRQHandler
   58 00000000                 IMPORT           EXTI9_5_IRQHandler
   59 00000000                 IMPORT           TIM1_BRK_IRQHandler
   60 00000000                 IMPORT           TIM1_UP_IRQHandler
   61 00000000                 IMPORT           TIM1_TRG_COM_IRQHandler
   62 00000000                 IMPORT           TIM1_CC_IRQHandler
   63 00000000                 IMPORT           TIM2_IRQHandler
   64 00000000                 IMPORT           TIM3_IRQHandler
   65 00000000                 IMPORT           TIM4_IRQHandler
   66 00000000                 IMPORT           I2C1_EV_IRQHandler
   67 00000000                 IMPORT           I2C1_ER_IRQHandler
   68 00000000                 IMPORT           I2C2_EV_IRQHandler
   69 00000000                 IMPORT           I2C2_ER_IRQHandler
   70 00000000                 IMPORT           SPI1_IRQHandler
   71 00000000                 IMPORT           SPI2_IRQHandler
   72 00000000                 IMPORT           USART1_IRQHandler
   73 00000000                 IMPORT           USART2_IRQHandler
   74 00000000                 IMPORT           USART3_IRQHandler
   75 00000000                 IMPORT           EXTI15_10_IRQHandler
   76 00000000                 IMPORT           RTCAlarm_IRQHandler
   77 00000000                 IMPORT           USBWakeUp_IRQHandler
   78 00000000                 IMPORT           TIM8_BRK_IRQHandler
   79 00000000                 IMPORT           TIM8_UP_IRQHandler
   80 00000000                 IMPORT           TIM8_TRG_COM_IRQHandler
   81 00000000                 IMPORT           TIM8_CC_IRQHandler
   82 00000000                 IMPORT           ADC3_IRQHandler
   83 00000000                 IMPORT           FSMC_IRQHandler
   84 00000000                 IMPORT           SDIO_IRQHandler
   85 00000000                 IMPORT           TIM5_IRQHandler
   86 00000000                 IMPORT           SPI3_IRQHandler
   87 00000000                 IMPORT           UART4_IRQHandler
   88 00000000                 IMPORT           UART5_IRQHandler
   89 00000000                 IMPORT           TIM6_IRQHandler
   90 00000000                 IMPORT           TIM7_IRQHandler
   91 00000000                 IMPORT           DMA2_Channel1_IRQHandler
   92 00000000                 IMPORT           DMA2_Channel2_IRQHandler
   93 00000000                 IMPORT           DMA2_Channel3_IRQHandler
   94 00000000                 IMPORT           DMA2_Channel4_5_IRQHandler
   95 00000000         
   96 00000000         ;IMPORT    SysTick_Handler    
   97 00000000                 IMPORT           uipPendSVHandler
   98 00000000                 IMPORT           uipSystemCounterHandler
   99 00000000         
  100 00000000 00000400 



ARM Macro Assembler    Page 3 


                       Stack_Size
                               EQU              0x00000400
  101 00000000         
  102 00000000                 AREA             STACK, NOINIT, READWRITE, ALIGN
=3
  103 00000000         Stack_Mem
                               SPACE            Stack_Size
  104 00000400         __initial_sp
  105 00000400         
  106 00000400         ; <h> Heap Configuration
  107 00000400         ;   <o>  Heap Size (in Bytes) <0x0-0xFFFFFFFF:8>
  108 00000400         ; </h>
  109 00000400         
  110 00000400 00000200 
                       Heap_Size
                               EQU              0x00000200
  111 00000400         
  112 00000400                 AREA             HEAP, NOINIT, READWRITE, ALIGN=
3
  113 00000000         __heap_base
  114 00000000         Heap_Mem
                               SPACE            Heap_Size
  115 00000200         __heap_limit
  116 00000200         
  117 00000200                 PRESERVE8
  118 00000200                 THUMB
  119 00000200         
  120 00000200         
  121 00000200         ; Vector Table Mapped to Address 0 at Reset
  122 00000200                 AREA             RESET, DATA, READONLY
  123 00000000                 EXPORT           __Vectors
  124 00000000                 EXPORT           __Vectors_End
  125 00000000                 EXPORT           __Vectors_Size
  126 00000000         
  127 00000000 00000000 
                       __Vectors
                               DCD              __initial_sp ; Top of Stack
  128 00000004 00000000        DCD              Reset_Handler ; Reset Handler
  129 00000008 00000000        DCD              NMI_Handler ; NMI Handler
  130 0000000C 00000000        DCD              HardFault_Handler ; Hard Fault 
                                                            Handler
  131 00000010 00000000        DCD              MemManage_Handler 
                                                            ; MPU Fault Handler
                                                            
  132 00000014 00000000        DCD              BusFault_Handler 
                                                            ; Bus Fault Handler
                                                            
  133 00000018 00000000        DCD              UsageFault_Handler ; Usage Faul
                                                            t Handler
  134 0000001C 00000000        DCD              0           ; Reserved
  135 00000020 00000000        DCD              0           ; Reserved
  136 00000024 00000000        DCD              0           ; Reserved
  137 00000028 00000000        DCD              0           ; Reserved
  138 0000002C 00000000        DCD              SVC_Handler ; SVCall Handler
  139 00000030 00000000        DCD              DebugMon_Handler ; Debug Monito
                                                            r Handler
  140 00000034 00000000        DCD              0           ; Reserved
  141 00000038 00000000        DCD              uipPendSVHandler 
                                                            ; PendSV Handler



ARM Macro Assembler    Page 4 


  142 0000003C 00000000        DCD              uipSystemCounterHandler 
                                                            ; SysTick Handler
  143 00000040         
  144 00000040         ; External Interrupts
  145 00000040 00000000        DCD              WWDG_IRQHandler 
                                                            ; Window Watchdog
  146 00000044 00000000        DCD              PVD_IRQHandler ; PVD through EX
                                                            TI Line detect
  147 00000048 00000000        DCD              TAMPER_IRQHandler ; Tamper
  148 0000004C 00000000        DCD              RTC_IRQHandler ; RTC
  149 00000050 00000000        DCD              FLASH_IRQHandler ; Flash
  150 00000054 00000000        DCD              RCC_IRQHandler ; RCC
  151 00000058 00000000        DCD              EXTI0_IRQHandler ; EXTI Line 0
  152 0000005C 00000000        DCD              EXTI1_IRQHandler ; EXTI Line 1
  153 00000060 00000000        DCD              EXTI2_IRQHandler ; EXTI Line 2
  154 00000064 00000000        DCD              EXTI3_IRQHandler ; EXTI Line 3
  155 00000068 00000000        DCD              EXTI4_IRQHandler ; EXTI Line 4
  156 0000006C 00000000        DCD              DMA1_Channel1_IRQHandler 
                                                            ; DMA1 Channel 1
  157 00000070 00000000        DCD              DMA1_Channel2_IRQHandler 
                                                            ; DMA1 Channel 2
  158 00000074 00000000        DCD              DMA1_Channel3_IRQHandler 
                                                            ; DMA1 Channel 3
  159 00000078 00000000        DCD              DMA1_Channel4_IRQHandler 
                                                            ; DMA1 Channel 4
  160 0000007C 00000000        DCD              DMA1_Channel5_IRQHandler 
                                                            ; DMA1 Channel 5
  161 00000080 00000000        DCD              DMA1_Channel6_IRQHandler 
                                                            ; DMA1 Channel 6
  162 00000084 00000000        DCD              DMA1_Channel7_IRQHandler 
                                                            ; DMA1 Channel 7
  163 00000088 00000000        DCD              ADC1_2_IRQHandler ; ADC1 & ADC2
                                                            
  164 0000008C 00000000        DCD              USB_HP_CAN1_TX_IRQHandler ; USB
                                                             High Priority or C
                                                            AN1 TX
  165 00000090 00000000        DCD              USB_LP_CAN1_RX0_IRQHandler ; US
                                                            B Low  Priority or 
                                                            CAN1 RX0
  166 00000094 00000000        DCD              CAN1_RX1_IRQHandler ; CAN1 RX1
  167 00000098 00000000        DCD              CAN1_SCE_IRQHandler ; CAN1 SCE
  168 0000009C 00000000        DCD              EXTI9_5_IRQHandler 
                                                            ; EXTI Line 9..5
  169 000000A0 00000000        DCD              TIM1_BRK_IRQHandler 
                                                            ; TIM1 Break
  170 000000A4 00000000        DCD              TIM1_UP_IRQHandler 
                                                            ; TIM1 Update
  171 000000A8 00000000        DCD              TIM1_TRG_COM_IRQHandler ; TIM1 
                                                            Trigger and Commuta
                                                            tion
  172 000000AC 00000000        DCD              TIM1_CC_IRQHandler ; TIM1 Captu
                                                            re Compare
  173 000000B0 00000000        DCD              TIM2_IRQHandler ; TIM2
  174 000000B4 00000000        DCD              TIM3_IRQHandler ; TIM3
  175 000000B8 00000000        DCD              TIM4_IRQHandler ; TIM4
  176 000000BC 00000000        DCD              I2C1_EV_IRQHandler ; I2C1 Event
                                                            
  177 000000C0 00000000        DCD              I2C1_ER_IRQHandler ; I2C1 Error
                                                            



ARM Macro Assembler    Page 5 


  178 000000C4 00000000        DCD              I2C2_EV_IRQHandler ; I2C2 Event
                                                            
  179 000000C8 00000000        DCD              I2C2_ER_IRQHandler ; I2C2 Error
                                                            
  180 000000CC 00000000        DCD              SPI1_IRQHandler ; SPI1
  181 000000D0 00000000        DCD              SPI2_IRQHandler ; SPI2
  182 000000D4 00000000        DCD              USART1_IRQHandler ; USART1
  183 000000D8 00000000        DCD              USART2_IRQHandler ; USART2
  184 000000DC 00000000        DCD              USART3_IRQHandler ; USART3
  185 000000E0 00000000        DCD              EXTI15_10_IRQHandler 
                                                            ; EXTI Line 15..10
  186 000000E4 00000000        DCD              RTCAlarm_IRQHandler ; RTC Alarm
                                                             through EXTI Line
  187 000000E8 00000000        DCD              USBWakeUp_IRQHandler ; USB Wake
                                                            up from suspend
  188 000000EC 00000000        DCD              TIM8_BRK_IRQHandler 
                                                            ; TIM8 Break
  189 000000F0 00000000        DCD              TIM8_UP_IRQHandler 
                                                            ; TIM8 Update
  190 000000F4 00000000        DCD              TIM8_TRG_COM_IRQHandler ; TIM8 
                                                            Trigger and Commuta
                                                            tion
  191 000000F8 00000000        DCD              TIM8_CC_IRQHandler ; TIM8 Captu
                                                            re Compare
  192 000000FC 00000000        DCD              ADC3_IRQHandler ; ADC3
  193 00000100 00000000        DCD              FSMC_IRQHandler ; FSMC
  194 00000104 00000000        DCD              SDIO_IRQHandler ; SDIO
  195 00000108 00000000        DCD              TIM5_IRQHandler ; TIM5
  196 0000010C 00000000        DCD              SPI3_IRQHandler ; SPI3
  197 00000110 00000000        DCD              UART4_IRQHandler ; UART4
  198 00000114 00000000        DCD              UART5_IRQHandler ; UART5
  199 00000118 00000000        DCD              TIM6_IRQHandler ; TIM6
  200 0000011C 00000000        DCD              TIM7_IRQHandler ; TIM7
  201 00000120 00000000        DCD              DMA2_Channel1_IRQHandler 
                                                            ; DMA2 Channel1
  202 00000124 00000000        DCD              DMA2_Channel2_IRQHandler 
                                                            ; DMA2 Channel2
  203 00000128 00000000        DCD              DMA2_Channel3_IRQHandler 
                                                            ; DMA2 Channel3
  204 0000012C 00000000        DCD              DMA2_Channel4_5_IRQHandler ; DM
                                                            A2 Channel4 & Chann
                                                            el5
  205 00000130         __Vectors_End
  206 00000130         
  207 00000130 00000130 
                       __Vectors_Size
                               EQU              __Vectors_End - __Vectors
  208 00000130         
  209 00000130                 AREA             |.text|, CODE, READONLY
  210 00000000         
  211 00000000         ; Reset handler
  212 00000000         Reset_Handler
                               PROC
  213 00000000                 EXPORT           Reset_Handler             [WEAK
]
  214 00000000                 IMPORT           __main
  215 00000000                 IMPORT           SystemInit
  216 00000000 4808            LDR              R0, =SystemInit
  217 00000002 4780            BLX              R0



ARM Macro Assembler    Page 6 


  218 00000004 4808            LDR              R0, =__main
  219 00000006 4700            BX               R0
  220 00000008                 ENDP
  221 00000008         
  222 00000008         ; Dummy Exception Handlers (infinite loops which can be 
                       modified)
  223 00000008         
  224 00000008         NMI_Handler
                               PROC
  225 00000008                 EXPORT           NMI_Handler                [WEA
K]
  226 00000008 E7FE            B                .
  227 0000000A                 ENDP
  229 0000000A         HardFault_Handler
                               PROC
  230 0000000A                 EXPORT           HardFault_Handler          [WEA
K]
  231 0000000A E7FE            B                .
  232 0000000C                 ENDP
  234 0000000C         MemManage_Handler
                               PROC
  235 0000000C                 EXPORT           MemManage_Handler          [WEA
K]
  236 0000000C E7FE            B                .
  237 0000000E                 ENDP
  239 0000000E         BusFault_Handler
                               PROC
  240 0000000E                 EXPORT           BusFault_Handler           [WEA
K]
  241 0000000E E7FE            B                .
  242 00000010                 ENDP
  244 00000010         UsageFault_Handler
                               PROC
  245 00000010                 EXPORT           UsageFault_Handler         [WEA
K]
  246 00000010 E7FE            B                .
  247 00000012                 ENDP
  248 00000012         SVC_Handler
                               PROC
  249 00000012                 EXPORT           SVC_Handler                [WEA
K]
  250 00000012 E7FE            B                .
  251 00000014                 ENDP
  253 00000014         DebugMon_Handler
                               PROC
  254 00000014                 EXPORT           DebugMon_Handler           [WEA
K]
  255 00000014 E7FE            B                .
  256 00000016                 ENDP
  257 00000016         
  258 00000016         Default_Handler
                               PROC
  259 00000016         
  260 00000016 E7FE            B                .
  261 00000018         
  262 00000018                 ENDP
  263 00000018         
  264 00000018                 ALIGN
  265 00000018         



ARM Macro Assembler    Page 7 


  266 00000018         ;*******************************************************
                       ************************
  267 00000018         ; User Stack and Heap initialization
  268 00000018         ;*******************************************************
                       ************************
  269 00000018                 IF               :DEF:__MICROLIB
  276 00000018         
  277 00000018                 IMPORT           __use_two_region_memory
  278 00000018                 EXPORT           __user_initial_stackheap
  279 00000018         
  280 00000018         __user_initial_stackheap
  281 00000018         
  282 00000018 4804            LDR              R0, =  Heap_Mem
  283 0000001A 4905            LDR              R1, =(Stack_Mem + Stack_Size)
  284 0000001C 4A05            LDR              R2, = (Heap_Mem +  Heap_Size)
  285 0000001E 4B06            LDR              R3, = Stack_Mem
  286 00000020 4770            BX               LR
  287 00000022         
  288 00000022 00 00           ALIGN
  289 00000024         
  290 00000024                 ENDIF
  291 00000024         
  292 00000024                 END
              00000000 
              00000000 
              00000000 
              00000400 
              00000200 
              00000000 
Command Line: --debug --xref --diag_suppress=9931 --cpu=Cortex-M3 --apcs=interw
ork --depend=.\objects\startup_stm32f10x_hd.d -o.\objects\startup_stm32f10x_hd.
o -IC:\Keil_v5\ARM\RV31\INC -IC:\Keil_v5\ARM\CMSIS\Include -IC:\Keil_v5\ARM\INC
\ST\STM32F10x --predefine="__UVISION_VERSION SETA 527" --list=.\listings\startu
p_stm32f10x_hd.lst startup\startup_stm32f10x_hd.s



ARM Macro Assembler    Page 1 Alphabetic symbol ordering
Relocatable symbols

STACK 00000000

Symbol: STACK
   Definitions
      At line 102 in file startup\startup_stm32f10x_hd.s
   Uses
      None
Comment: STACK unused
Stack_Mem 00000000

Symbol: Stack_Mem
   Definitions
      At line 103 in file startup\startup_stm32f10x_hd.s
   Uses
      At line 283 in file startup\startup_stm32f10x_hd.s
      At line 285 in file startup\startup_stm32f10x_hd.s

__initial_sp 00000400

Symbol: __initial_sp
   Definitions
      At line 104 in file startup\startup_stm32f10x_hd.s
   Uses
      At line 127 in file startup\startup_stm32f10x_hd.s
Comment: __initial_sp used once
3 symbols



ARM Macro Assembler    Page 1 Alphabetic symbol ordering
Relocatable symbols

HEAP 00000000

Symbol: HEAP
   Definitions
      At line 112 in file startup\startup_stm32f10x_hd.s
   Uses
      None
Comment: HEAP unused
Heap_Mem 00000000

Symbol: Heap_Mem
   Definitions
      At line 114 in file startup\startup_stm32f10x_hd.s
   Uses
      At line 282 in file startup\startup_stm32f10x_hd.s
      At line 284 in file startup\startup_stm32f10x_hd.s

__heap_base 00000000

Symbol: __heap_base
   Definitions
      At line 113 in file startup\startup_stm32f10x_hd.s
   Uses
      None
Comment: __heap_base unused
__heap_limit 00000200

Symbol: __heap_limit
   Definitions
      At line 115 in file startup\startup_stm32f10x_hd.s
   Uses
      None
Comment: __heap_limit unused
4 symbols



ARM Macro Assembler    Page 1 Alphabetic symbol ordering
Relocatable symbols

RESET 00000000

Symbol: RESET
   Definitions
      At line 122 in file startup\startup_stm32f10x_hd.s
   Uses
      None
Comment: RESET unused
__Vectors 00000000

Symbol: __Vectors
   Definitions
      At line 127 in file startup\startup_stm32f10x_hd.s
   Uses
      At line 123 in file startup\startup_stm32f10x_hd.s
      At line 207 in file startup\startup_stm32f10x_hd.s

__Vectors_End 00000130

Symbol: __Vectors_End
   Definitions
      At line 205 in file startup\startup_stm32f10x_hd.s
   Uses
      At line 124 in file startup\startup_stm32f10x_hd.s
      At line 207 in file startup\startup_stm32f10x_hd.s

3 symbols



ARM Macro Assembler    Page 1 Alphabetic symbol ordering
Relocatable symbols

.text 00000000

Symbol: .text
   Definitions
      At line 209 in file startup\startup_stm32f10x_hd.s
   Uses
      None
Comment: .text unused
BusFault_Handler 0000000E

Symbol: BusFault_Handler
   Definitions
      At line 239 in file startup\startup_stm32f10x_hd.s
   Uses
      At line 132 in file startup\startup_stm32f10x_hd.s
      At line 240 in file startup\startup_stm32f10x_hd.s

DebugMon_Handler 00000014

Symbol: DebugMon_Handler
   Definitions
      At line 253 in file startup\startup_stm32f10x_hd.s
   Uses
      At line 139 in file startup\startup_stm32f10x_hd.s
      At line 254 in file startup\startup_stm32f10x_hd.s

Default_Handler 00000016

Symbol: Default_Handler
   Definitions
      At line 258 in file startup\startup_stm32f10x_hd.s
   Uses
      None
Comment: Default_Handler unused
HardFault_Handler 0000000A

Symbol: HardFault_Handler
   Definitions
      At line 229 in file startup\startup_stm32f10x_hd.s
   Uses
      At line 130 in file startup\startup_stm32f10x_hd.s
      At line 230 in file startup\startup_stm32f10x_hd.s

MemManage_Handler 0000000C

Symbol: MemManage_Handler
   Definitions
      At line 234 in file startup\startup_stm32f10x_hd.s
   Uses
      At line 131 in file startup\startup_stm32f10x_hd.s
      At line 235 in file startup\startup_stm32f10x_hd.s

NMI_Handler 00000008

Symbol: NMI_Handler
   Definitions
      At line 224 in file startup\startup_stm32f10x_hd.s
   Uses
      At line 129 in file startup\startup_stm32f10x_hd.s



ARM Macro Assembler    Page 2 Alphabetic symbol ordering
Relocatable symbols

      At line 225 in file startup\startup_stm32f10x_hd.s

Reset_Handler 00000000

Symbol: Reset_Handler
   Definitions
      At line 212 in file startup\startup_stm32f10x_hd.s
   Uses
      At line 128 in file startup\startup_stm32f10x_hd.s
      At line 213 in file startup\startup_stm32f10x_hd.s

SVC_Handler 00000012

Symbol: SVC_Handler
   Definitions
      At line 248 in file startup\startup_stm32f10x_hd.s
   Uses
      At line 138 in file startup\startup_stm32f10x_hd.s
      At line 249 in file startup\startup_stm32f10x_hd.s

UsageFault_Handler 00000010

Symbol: UsageFault_Handler
   Definitions
      At line 244 in file startup\startup_stm32f10x_hd.s
   Uses
      At line 133 in file startup\startup_stm32f10x_hd.s
      At line 245 in file startup\startup_stm32f10x_hd.s

__user_initial_stackheap 00000018

Symbol: __user_initial_stackheap
   Definitions
      At line 280 in file startup\startup_stm32f10x_hd.s
   Uses
      At line 278 in file startup\startup_stm32f10x_hd.s
Comment: __user_initial_stackheap used once
11 symbols



ARM Macro Assembler    Page 1 Alphabetic symbol ordering
Absolute symbols

Heap_Size 00000200

Symbol: Heap_Size
   Definitions
      At line 110 in file startup\startup_stm32f10x_hd.s
   Uses
      At line 114 in file startup\startup_stm32f10x_hd.s
      At line 284 in file startup\startup_stm32f10x_hd.s

Stack_Size 00000400

Symbol: Stack_Size
   Definitions
      At line 100 in file startup\startup_stm32f10x_hd.s
   Uses
      At line 103 in file startup\startup_stm32f10x_hd.s
      At line 283 in file startup\startup_stm32f10x_hd.s

__Vectors_Size 00000130

Symbol: __Vectors_Size
   Definitions
      At line 207 in file startup\startup_stm32f10x_hd.s
   Uses
      At line 125 in file startup\startup_stm32f10x_hd.s
Comment: __Vectors_Size used once
3 symbols



ARM Macro Assembler    Page 1 Alphabetic symbol ordering
External symbols

ADC1_2_IRQHandler 00000000

Symbol: ADC1_2_IRQHandler
   Definitions
      At line 53 in file startup\startup_stm32f10x_hd.s
   Uses
      At line 163 in file startup\startup_stm32f10x_hd.s
Comment: ADC1_2_IRQHandler used once
ADC3_IRQHandler 00000000

Symbol: ADC3_IRQHandler
   Definitions
      At line 82 in file startup\startup_stm32f10x_hd.s
   Uses
      At line 192 in file startup\startup_stm32f10x_hd.s
Comment: ADC3_IRQHandler used once
CAN1_RX1_IRQHandler 00000000

Symbol: CAN1_RX1_IRQHandler
   Definitions
      At line 56 in file startup\startup_stm32f10x_hd.s
   Uses
      At line 166 in file startup\startup_stm32f10x_hd.s
Comment: CAN1_RX1_IRQHandler used once
CAN1_SCE_IRQHandler 00000000

Symbol: CAN1_SCE_IRQHandler
   Definitions
      At line 57 in file startup\startup_stm32f10x_hd.s
   Uses
      At line 167 in file startup\startup_stm32f10x_hd.s
Comment: CAN1_SCE_IRQHandler used once
DMA1_Channel1_IRQHandler 00000000

Symbol: DMA1_Channel1_IRQHandler
   Definitions
      At line 46 in file startup\startup_stm32f10x_hd.s
   Uses
      At line 156 in file startup\startup_stm32f10x_hd.s
Comment: DMA1_Channel1_IRQHandler used once
DMA1_Channel2_IRQHandler 00000000

Symbol: DMA1_Channel2_IRQHandler
   Definitions
      At line 47 in file startup\startup_stm32f10x_hd.s
   Uses
      At line 157 in file startup\startup_stm32f10x_hd.s
Comment: DMA1_Channel2_IRQHandler used once
DMA1_Channel3_IRQHandler 00000000

Symbol: DMA1_Channel3_IRQHandler
   Definitions
      At line 48 in file startup\startup_stm32f10x_hd.s
   Uses
      At line 158 in file startup\startup_stm32f10x_hd.s
Comment: DMA1_Channel3_IRQHandler used once
DMA1_Channel4_IRQHandler 00000000

Symbol: DMA1_Channel4_IRQHandler



ARM Macro Assembler    Page 2 Alphabetic symbol ordering
External symbols

   Definitions
      At line 49 in file startup\startup_stm32f10x_hd.s
   Uses
      At line 159 in file startup\startup_stm32f10x_hd.s
Comment: DMA1_Channel4_IRQHandler used once
DMA1_Channel5_IRQHandler 00000000

Symbol: DMA1_Channel5_IRQHandler
   Definitions
      At line 50 in file startup\startup_stm32f10x_hd.s
   Uses
      At line 160 in file startup\startup_stm32f10x_hd.s
Comment: DMA1_Channel5_IRQHandler used once
DMA1_Channel6_IRQHandler 00000000

Symbol: DMA1_Channel6_IRQHandler
   Definitions
      At line 51 in file startup\startup_stm32f10x_hd.s
   Uses
      At line 161 in file startup\startup_stm32f10x_hd.s
Comment: DMA1_Channel6_IRQHandler used once
DMA1_Channel7_IRQHandler 00000000

Symbol: DMA1_Channel7_IRQHandler
   Definitions
      At line 52 in file startup\startup_stm32f10x_hd.s
   Uses
      At line 162 in file startup\startup_stm32f10x_hd.s
Comment: DMA1_Channel7_IRQHandler used once
DMA2_Channel1_IRQHandler 00000000

Symbol: DMA2_Channel1_IRQHandler
   Definitions
      At line 91 in file startup\startup_stm32f10x_hd.s
   Uses
      At line 201 in file startup\startup_stm32f10x_hd.s
Comment: DMA2_Channel1_IRQHandler used once
DMA2_Channel2_IRQHandler 00000000

Symbol: DMA2_Channel2_IRQHandler
   Definitions
      At line 92 in file startup\startup_stm32f10x_hd.s
   Uses
      At line 202 in file startup\startup_stm32f10x_hd.s
Comment: DMA2_Channel2_IRQHandler used once
DMA2_Channel3_IRQHandler 00000000

Symbol: DMA2_Channel3_IRQHandler
   Definitions
      At line 93 in file startup\startup_stm32f10x_hd.s
   Uses
      At line 203 in file startup\startup_stm32f10x_hd.s
Comment: DMA2_Channel3_IRQHandler used once
DMA2_Channel4_5_IRQHandler 00000000

Symbol: DMA2_Channel4_5_IRQHandler
   Definitions
      At line 94 in file startup\startup_stm32f10x_hd.s
   Uses



ARM Macro Assembler    Page 3 Alphabetic symbol ordering
External symbols

      At line 204 in file startup\startup_stm32f10x_hd.s
Comment: DMA2_Channel4_5_IRQHandler used once
EXTI0_IRQHandler 00000000

Symbol: EXTI0_IRQHandler
   Definitions
      At line 41 in file startup\startup_stm32f10x_hd.s
   Uses
      At line 151 in file startup\startup_stm32f10x_hd.s
Comment: EXTI0_IRQHandler used once
EXTI15_10_IRQHandler 00000000

Symbol: EXTI15_10_IRQHandler
   Definitions
      At line 75 in file startup\startup_stm32f10x_hd.s
   Uses
      At line 185 in file startup\startup_stm32f10x_hd.s
Comment: EXTI15_10_IRQHandler used once
EXTI1_IRQHandler 00000000

Symbol: EXTI1_IRQHandler
   Definitions
      At line 42 in file startup\startup_stm32f10x_hd.s
   Uses
      At line 152 in file startup\startup_stm32f10x_hd.s
Comment: EXTI1_IRQHandler used once
EXTI2_IRQHandler 00000000

Symbol: EXTI2_IRQHandler
   Definitions
      At line 43 in file startup\startup_stm32f10x_hd.s
   Uses
      At line 153 in file startup\startup_stm32f10x_hd.s
Comment: EXTI2_IRQHandler used once
EXTI3_IRQHandler 00000000

Symbol: EXTI3_IRQHandler
   Definitions
      At line 44 in file startup\startup_stm32f10x_hd.s
   Uses
      At line 154 in file startup\startup_stm32f10x_hd.s
Comment: EXTI3_IRQHandler used once
EXTI4_IRQHandler 00000000

Symbol: EXTI4_IRQHandler
   Definitions
      At line 45 in file startup\startup_stm32f10x_hd.s
   Uses
      At line 155 in file startup\startup_stm32f10x_hd.s
Comment: EXTI4_IRQHandler used once
EXTI9_5_IRQHandler 00000000

Symbol: EXTI9_5_IRQHandler
   Definitions
      At line 58 in file startup\startup_stm32f10x_hd.s
   Uses
      At line 168 in file startup\startup_stm32f10x_hd.s
Comment: EXTI9_5_IRQHandler used once
FLASH_IRQHandler 00000000



ARM Macro Assembler    Page 4 Alphabetic symbol ordering
External symbols


Symbol: FLASH_IRQHandler
   Definitions
      At line 39 in file startup\startup_stm32f10x_hd.s
   Uses
      At line 149 in file startup\startup_stm32f10x_hd.s
Comment: FLASH_IRQHandler used once
FSMC_IRQHandler 00000000

Symbol: FSMC_IRQHandler
   Definitions
      At line 83 in file startup\startup_stm32f10x_hd.s
   Uses
      At line 193 in file startup\startup_stm32f10x_hd.s
Comment: FSMC_IRQHandler used once
I2C1_ER_IRQHandler 00000000

Symbol: I2C1_ER_IRQHandler
   Definitions
      At line 67 in file startup\startup_stm32f10x_hd.s
   Uses
      At line 177 in file startup\startup_stm32f10x_hd.s
Comment: I2C1_ER_IRQHandler used once
I2C1_EV_IRQHandler 00000000

Symbol: I2C1_EV_IRQHandler
   Definitions
      At line 66 in file startup\startup_stm32f10x_hd.s
   Uses
      At line 176 in file startup\startup_stm32f10x_hd.s
Comment: I2C1_EV_IRQHandler used once
I2C2_ER_IRQHandler 00000000

Symbol: I2C2_ER_IRQHandler
   Definitions
      At line 69 in file startup\startup_stm32f10x_hd.s
   Uses
      At line 179 in file startup\startup_stm32f10x_hd.s
Comment: I2C2_ER_IRQHandler used once
I2C2_EV_IRQHandler 00000000

Symbol: I2C2_EV_IRQHandler
   Definitions
      At line 68 in file startup\startup_stm32f10x_hd.s
   Uses
      At line 178 in file startup\startup_stm32f10x_hd.s
Comment: I2C2_EV_IRQHandler used once
PVD_IRQHandler 00000000

Symbol: PVD_IRQHandler
   Definitions
      At line 36 in file startup\startup_stm32f10x_hd.s
   Uses
      At line 146 in file startup\startup_stm32f10x_hd.s
Comment: PVD_IRQHandler used once
RCC_IRQHandler 00000000

Symbol: RCC_IRQHandler
   Definitions



ARM Macro Assembler    Page 5 Alphabetic symbol ordering
External symbols

      At line 40 in file startup\startup_stm32f10x_hd.s
   Uses
      At line 150 in file startup\startup_stm32f10x_hd.s
Comment: RCC_IRQHandler used once
RTCAlarm_IRQHandler 00000000

Symbol: RTCAlarm_IRQHandler
   Definitions
      At line 76 in file startup\startup_stm32f10x_hd.s
   Uses
      At line 186 in file startup\startup_stm32f10x_hd.s
Comment: RTCAlarm_IRQHandler used once
RTC_IRQHandler 00000000

Symbol: RTC_IRQHandler
   Definitions
      At line 38 in file startup\startup_stm32f10x_hd.s
   Uses
      At line 148 in file startup\startup_stm32f10x_hd.s
Comment: RTC_IRQHandler used once
SDIO_IRQHandler 00000000

Symbol: SDIO_IRQHandler
   Definitions
      At line 84 in file startup\startup_stm32f10x_hd.s
   Uses
      At line 194 in file startup\startup_stm32f10x_hd.s
Comment: SDIO_IRQHandler used once
SPI1_IRQHandler 00000000

Symbol: SPI1_IRQHandler
   Definitions
      At line 70 in file startup\startup_stm32f10x_hd.s
   Uses
      At line 180 in file startup\startup_stm32f10x_hd.s
Comment: SPI1_IRQHandler used once
SPI2_IRQHandler 00000000

Symbol: SPI2_IRQHandler
   Definitions
      At line 71 in file startup\startup_stm32f10x_hd.s
   Uses
      At line 181 in file startup\startup_stm32f10x_hd.s
Comment: SPI2_IRQHandler used once
SPI3_IRQHandler 00000000

Symbol: SPI3_IRQHandler
   Definitions
      At line 86 in file startup\startup_stm32f10x_hd.s
   Uses
      At line 196 in file startup\startup_stm32f10x_hd.s
Comment: SPI3_IRQHandler used once
SystemInit 00000000

Symbol: SystemInit
   Definitions
      At line 215 in file startup\startup_stm32f10x_hd.s
   Uses
      At line 216 in file startup\startup_stm32f10x_hd.s



ARM Macro Assembler    Page 6 Alphabetic symbol ordering
External symbols

Comment: SystemInit used once
TAMPER_IRQHandler 00000000

Symbol: TAMPER_IRQHandler
   Definitions
      At line 37 in file startup\startup_stm32f10x_hd.s
   Uses
      At line 147 in file startup\startup_stm32f10x_hd.s
Comment: TAMPER_IRQHandler used once
TIM1_BRK_IRQHandler 00000000

Symbol: TIM1_BRK_IRQHandler
   Definitions
      At line 59 in file startup\startup_stm32f10x_hd.s
   Uses
      At line 169 in file startup\startup_stm32f10x_hd.s
Comment: TIM1_BRK_IRQHandler used once
TIM1_CC_IRQHandler 00000000

Symbol: TIM1_CC_IRQHandler
   Definitions
      At line 62 in file startup\startup_stm32f10x_hd.s
   Uses
      At line 172 in file startup\startup_stm32f10x_hd.s
Comment: TIM1_CC_IRQHandler used once
TIM1_TRG_COM_IRQHandler 00000000

Symbol: TIM1_TRG_COM_IRQHandler
   Definitions
      At line 61 in file startup\startup_stm32f10x_hd.s
   Uses
      At line 171 in file startup\startup_stm32f10x_hd.s
Comment: TIM1_TRG_COM_IRQHandler used once
TIM1_UP_IRQHandler 00000000

Symbol: TIM1_UP_IRQHandler
   Definitions
      At line 60 in file startup\startup_stm32f10x_hd.s
   Uses
      At line 170 in file startup\startup_stm32f10x_hd.s
Comment: TIM1_UP_IRQHandler used once
TIM2_IRQHandler 00000000

Symbol: TIM2_IRQHandler
   Definitions
      At line 63 in file startup\startup_stm32f10x_hd.s
   Uses
      At line 173 in file startup\startup_stm32f10x_hd.s
Comment: TIM2_IRQHandler used once
TIM3_IRQHandler 00000000

Symbol: TIM3_IRQHandler
   Definitions
      At line 64 in file startup\startup_stm32f10x_hd.s
   Uses
      At line 174 in file startup\startup_stm32f10x_hd.s
Comment: TIM3_IRQHandler used once
TIM4_IRQHandler 00000000




ARM Macro Assembler    Page 7 Alphabetic symbol ordering
External symbols

Symbol: TIM4_IRQHandler
   Definitions
      At line 65 in file startup\startup_stm32f10x_hd.s
   Uses
      At line 175 in file startup\startup_stm32f10x_hd.s
Comment: TIM4_IRQHandler used once
TIM5_IRQHandler 00000000

Symbol: TIM5_IRQHandler
   Definitions
      At line 85 in file startup\startup_stm32f10x_hd.s
   Uses
      At line 195 in file startup\startup_stm32f10x_hd.s
Comment: TIM5_IRQHandler used once
TIM6_IRQHandler 00000000

Symbol: TIM6_IRQHandler
   Definitions
      At line 89 in file startup\startup_stm32f10x_hd.s
   Uses
      At line 199 in file startup\startup_stm32f10x_hd.s
Comment: TIM6_IRQHandler used once
TIM7_IRQHandler 00000000

Symbol: TIM7_IRQHandler
   Definitions
      At line 90 in file startup\startup_stm32f10x_hd.s
   Uses
      At line 200 in file startup\startup_stm32f10x_hd.s
Comment: TIM7_IRQHandler used once
TIM8_BRK_IRQHandler 00000000

Symbol: TIM8_BRK_IRQHandler
   Definitions
      At line 78 in file startup\startup_stm32f10x_hd.s
   Uses
      At line 188 in file startup\startup_stm32f10x_hd.s
Comment: TIM8_BRK_IRQHandler used once
TIM8_CC_IRQHandler 00000000

Symbol: TIM8_CC_IRQHandler
   Definitions
      At line 81 in file startup\startup_stm32f10x_hd.s
   Uses
      At line 191 in file startup\startup_stm32f10x_hd.s
Comment: TIM8_CC_IRQHandler used once
TIM8_TRG_COM_IRQHandler 00000000

Symbol: TIM8_TRG_COM_IRQHandler
   Definitions
      At line 80 in file startup\startup_stm32f10x_hd.s
   Uses
      At line 190 in file startup\startup_stm32f10x_hd.s
Comment: TIM8_TRG_COM_IRQHandler used once
TIM8_UP_IRQHandler 00000000

Symbol: TIM8_UP_IRQHandler
   Definitions
      At line 79 in file startup\startup_stm32f10x_hd.s



ARM Macro Assembler    Page 8 Alphabetic symbol ordering
External symbols

   Uses
      At line 189 in file startup\startup_stm32f10x_hd.s
Comment: TIM8_UP_IRQHandler used once
UART4_IRQHandler 00000000

Symbol: UART4_IRQHandler
   Definitions
      At line 87 in file startup\startup_stm32f10x_hd.s
   Uses
      At line 197 in file startup\startup_stm32f10x_hd.s
Comment: UART4_IRQHandler used once
UART5_IRQHandler 00000000

Symbol: UART5_IRQHandler
   Definitions
      At line 88 in file startup\startup_stm32f10x_hd.s
   Uses
      At line 198 in file startup\startup_stm32f10x_hd.s
Comment: UART5_IRQHandler used once
USART1_IRQHandler 00000000

Symbol: USART1_IRQHandler
   Definitions
      At line 72 in file startup\startup_stm32f10x_hd.s
   Uses
      At line 182 in file startup\startup_stm32f10x_hd.s
Comment: USART1_IRQHandler used once
USART2_IRQHandler 00000000

Symbol: USART2_IRQHandler
   Definitions
      At line 73 in file startup\startup_stm32f10x_hd.s
   Uses
      At line 183 in file startup\startup_stm32f10x_hd.s
Comment: USART2_IRQHandler used once
USART3_IRQHandler 00000000

Symbol: USART3_IRQHandler
   Definitions
      At line 74 in file startup\startup_stm32f10x_hd.s
   Uses
      At line 184 in file startup\startup_stm32f10x_hd.s
Comment: USART3_IRQHandler used once
USBWakeUp_IRQHandler 00000000

Symbol: USBWakeUp_IRQHandler
   Definitions
      At line 77 in file startup\startup_stm32f10x_hd.s
   Uses
      At line 187 in file startup\startup_stm32f10x_hd.s
Comment: USBWakeUp_IRQHandler used once
USB_HP_CAN1_TX_IRQHandler 00000000

Symbol: USB_HP_CAN1_TX_IRQHandler
   Definitions
      At line 54 in file startup\startup_stm32f10x_hd.s
   Uses
      At line 164 in file startup\startup_stm32f10x_hd.s
Comment: USB_HP_CAN1_TX_IRQHandler used once



ARM Macro Assembler    Page 9 Alphabetic symbol ordering
External symbols

USB_LP_CAN1_RX0_IRQHandler 00000000

Symbol: USB_LP_CAN1_RX0_IRQHandler
   Definitions
      At line 55 in file startup\startup_stm32f10x_hd.s
   Uses
      At line 165 in file startup\startup_stm32f10x_hd.s
Comment: USB_LP_CAN1_RX0_IRQHandler used once
WWDG_IRQHandler 00000000

Symbol: WWDG_IRQHandler
   Definitions
      At line 35 in file startup\startup_stm32f10x_hd.s
   Uses
      At line 145 in file startup\startup_stm32f10x_hd.s
Comment: WWDG_IRQHandler used once
__main 00000000

Symbol: __main
   Definitions
      At line 214 in file startup\startup_stm32f10x_hd.s
   Uses
      At line 218 in file startup\startup_stm32f10x_hd.s
Comment: __main used once
__use_two_region_memory 00000000

Symbol: __use_two_region_memory
   Definitions
      At line 277 in file startup\startup_stm32f10x_hd.s
   Uses
      None
Comment: __use_two_region_memory unused
uipPendSVHandler 00000000

Symbol: uipPendSVHandler
   Definitions
      At line 97 in file startup\startup_stm32f10x_hd.s
   Uses
      At line 141 in file startup\startup_stm32f10x_hd.s
Comment: uipPendSVHandler used once
uipSystemCounterHandler 00000000

Symbol: uipSystemCounterHandler
   Definitions
      At line 98 in file startup\startup_stm32f10x_hd.s
   Uses
      At line 142 in file startup\startup_stm32f10x_hd.s
Comment: uipSystemCounterHandler used once
65 symbols
424 symbols in table
